:100000000C94C1000C944F020C94DE000C94DE00A2
:100010000C94DE000C94DE000C94DE000C94DE00E8
:100020000C94DE000C94DE000C94DE000C94DE00D8
:100030000C94DE000C94DE000C94DE000C94DE00C8
:100040000C94DE000C94DE000C94DE000C94DE00B8
:100050000C94DE000C94DE000C94DE000C94DE00A8
:100060000C94DE000C94DE005A0B680B6C0B700BCA
:10007000740B780B7C0B800B840B880B1C035700D4
:100080005500530042006D006F00740065005F0072
:10009000760031002E0032001803720061007000FB
:1000A00068006E00650074002E006E00650074002C
:1000B0000403090405010905A1010901A100093092
:1000C0000931150026FF00750895028102093309E0
:1000D000340935150026FF03750A95038102750161
:1000E00095028103C0050919012910150025017524
:1000F0000195108102C0A1020600FF09011500262A
:10010000FF0075089505B100C01201010100000053
:10011000089B2810000201010203011201010100E5
:100120000000089B281100020101020301050109DA
:1001300002A1010901A100050919012904150025E1
:10014000019504750181029501750481030501097A
:100150003009311581257F750895028106158125A5
:100160007F350045000938750895018106C0C0A19A
:10017000020600FF0901150026FF0075089505B16C
:1001800000C011241FBECFEFD4E0DEBFCDBF11E011
:10019000A0E0B1E0EEE2F9E102C005900D92A835D1
:1001A000B107D9F711E0A8E5B1E001C01D92AA3E60
:1001B000B107E1F70E94950B0C94950C0C9400008C
:1001C000CF93C62F2091AE0124FF07C02091AF012D
:1001D00038E823272093AF0103C02AE52093AE011E
:1001E000DC01E0EBF1E09C2F9E0F8D918193892F34
:1001F0008E1B1816D4F36C2F80EB91E00E944B02FB
:10020000CC5FC093AE01CF910895CF93DF936091FF
:10021000BF01635067FDC5C08091BC01CCE0D0E058
:10022000C81BD109CD53DE4F8091BB018D3209F03F
:10023000A6C0683009F0B3C083EC8093A3018AE5BF
:1002400080930101109258018881807621F0CE01BF
:100250000E94B70381C09A811092AC0189818111FB
:1002600006C01092AD012CEA31E082E071C0853009
:1002700019F49093C00169C0863009F050C08B8199
:10028000813009F442C0823029F4CE010E948903F2
:1002900090E042C0833061F5911109C080EB90E09D
:1002A0009093BE018093BD0190E484E035C091300D
:1002B00049F488E990E09093BE018093BD0190E4F9
:1002C00088E12AC0923049F48CE790E09093BE0117
:1002D0008093BD0190E48CE11FC09330D9F48EE48B
:1002E00091E09093BE018093BD0190E08CE014C03A
:1002F000813249F48BE691E09093BE018093BD0179
:1003000090E489E009C0823229F4CE010E94890379
:1003100090E402C090E480E0909358011DC08830C2
:1003200069F0893019F49093C2010FC08A3049F006
:100330008B3059F48BE48093AF0107C022EC31E09D
:1003400002C02CEA31E081E003C02CEA31E080E019
:100350003093BE012093BD018F3F39F4988197FD02
:100360008E8190E89093580107C09F81911104C03D
:100370009E81981708F4892F8093000110C0809106
:10038000580187FF0CC0CE010E94FF038F3F21F46C
:100390008EE18093010103C081111092000110923F
:1003A000BF018091010184FF47C0809100018F3F10
:1003B00009F442C0C82F893008F0C8E08C1B809334
:1003C00000018091A30198E889278093A301CC23A1
:1003D00031F12091BD013091BE018091580186FF1D
:1003E0000BC0A4EAB1E0F9018C2F8A0F94919D9380
:1003F00031968A13FBCF09C0D901E4EAF1E08C2FD2
:100400008E0F9D9191938E13FCCF8FEF8C0F90E008
:100410000196820F931F9093BE018093BD016C2FB4
:1004200084EA91E00E944B02CC5FCC3019F08FEF50
:1004300080930001C093010184E199B1957031F47A
:100440008150D9F71092C0011092BA01DF91CF917B
:100450000895E9E6F0E0808182608083E89A8BE489
:100460008093AF018AE58093AE010895A82FB92F3C
:1004700080E090E041E050EA609530E009C02D91C5
:1004800082279795879510F084279527305EC8F3CB
:100490006F5FA8F30895EADF8D939D930895CF933E
:1004A000CFB7CF93C395489BE9F7489B09C0489BBA
:1004B00007C0489B05C0489B03C0489B01C0A3C020
:1004C000DF93C091BC01DD27CD53DE4F489B02C0B6
:1004D000DF91EBCF2F930F931F9309B12FEF00FB09
:1004E00020F94F933F9319B14FEF012700FB21F9FA
:1004F0003BE031C04E7F012F19B1216028C0102F81
:100500004D7F2260000009B129C04B7F2460012F7C
:10051000000019B12BC019B1477F28602AC04F7E57
:1005200009B120612CC04F7D19B120622FC04F7BD3
:1005300009B1206432C0422709B149934FEF00004E
:10054000102710FB20F919B11570C9F1297F91F21C
:10055000012700FB21F909B1237F89F2315058F1BD
:10056000102710FB22F919B1277E79F2012700FB31
:1005700023F92F7C81F209B1102710FB24F92F7980
:1005800071F200C019B1012700FB25F92F7359F250
:1005900000C009B1102710FB26F9223040F200C03C
:1005A00019B1012700FB27F9243028F64F7720687E
:1005B00019B10000F9CF11E01CBB002719C03B5056
:1005C0003195C31BD04011E01CBB0881033CF9F0FE
:1005D0000B34E9F02091BA011981110F1213EDCFFC
:1005E0004A81441F093641F10D3211F0013E29F7CD
:1005F0000093C1013F914F911F910F912F91DF9176
:10060000CCB3C0FD4FCFCF91CFBFCF9118952091E4
:10061000C101222379F31091BF01112369F5343010
:100620006AF13093BF012093BB011091BC013BE004
:10063000311B3093BC0122C00091BF010130E4F4B2
:100640000AE54F7049F43091010134FD19C000935F
:100650000101C3EAD1E018C03091AE0134FD10C0F1
:100660000093AE01CFEAD1E00FC02795A8F4515016
:10067000A9F4220F0000F9CF4AE503C042ED01C002
:10068000432FC4E1D0E032E01AB11560589A1AB98C
:100690000BB120E415E05F93012756E00BB92795D5
:1006A00020F4515021F4220FF9CF012756E0000029
:1006B0003B5A0BB9D0F2279528F4515029F4220F58
:1006C0000000F9CF012756E027950BB920F45150CF
:1006D00021F4220FF9CF012756E0299133230BB9DA
:1006E00021F60A7F1091C001110FC651D0400BB9FD
:1006F00011F01093BA0111E01CBB01601AB11A7F0E
:10070000402F4A7F5F9100C000C00BB91AB94BB9A6
:1007100071CFFC018081807641F59181963031F571
:1007200093819230D1F0923269F09130F9F4809156
:100730006F01909170019093BE018093BD018091F3
:100740006E01089580917201909173019093BE01A2
:100750008093BD0180917101089582E091E09093B2
:10076000BE018093BD0182E2089580E00895CF9399
:10077000DF9300D000D0CDB7DEB7FC0182E691E078
:100780009093BE018093BD01808180768032C1F05C
:10079000803469F58281898383818A8384818B8314
:1007A00085818C838AE591E09093BE018093BD01A1
:1007B000AC01BE016F5F7F4F81810E944B0B18C05F
:1007C0008181813021F0893091F48FEF11C0E09167
:1007D0006C01F0916D010088F189E02D82E691E0D5
:1007E0000995E0916C01F0916D01808101C080E07C
:1007F0000F900F900F900F90DF91CF910895CF93AE
:10080000DF93CDB7DEB728970FB6F894DEBF0FBEE3
:10081000CDBF653011F08FEF0DC0BC016F5F7F4F12
:10082000AE014F5F5F4FFC0180810E944B0B88231C
:1008300091F381E028960FB6F894DEBF0FBECDBFCE
:10084000DF91CF910895EF92FF920F931F93CF9373
:10085000DF93E0916C01F0916D01008111810088BE
:10086000F189E02D82E691E00995C0E0D0E07801C1
:10087000EC1AFD0AE0916C01F0916D01808191818B
:100880008C179D07ACF08091AE0184FD04C00E94DE
:100890000501A895F8CFB7016930710514F068E03B
:1008A00070E0CE018E599E4F0E94E0002896DFCF67
:1008B000DF91CF911F910F91FF90EF9008950097D6
:1008C00041F028E0E9E8F1E0DC0101900D922A9581
:1008D000E1F788E0E9E8F1E0A1E8B1E001900D92EC
:1008E0008A95E1F70895EF920F931F93CF93DF93CB
:1008F00000D0CDB7DEB769834A83E12C00E010E079
:1009000020E030E0AE014F5F5F4F62E070E00E9498
:10091000FD09EFEAF4E03197F1F700C000000F9015
:100920000F90DF91CF911F910F91EF9008958091DB
:10093000240190912501892B31F01092250110920C
:10094000240181E0089548E050E061E871E089E821
:1009500091E00E94560C0895AF92BF92CF92DF9221
:10096000EF920F931F93CF93DF931F92CDB7DEB714
:1009700089835B016A01E12C00E010E020E030E0B7
:10098000AE014F5F5F4F61E070E082E50E94FD09BC
:10099000811117C08FEA94E00197F1F700C00000C1
:1009A0008501960140E050E060E070E082E50E9441
:1009B000FD09811106C0EFEAF4E03197F1F700C0BC
:1009C00000000F90DF91CF911F910F91EF90DF907A
:1009D000CF90BF90AF9008950F931F93CF93DF9365
:1009E000CDB7DEB760970FB6F894DEBF0FBECDBFB0
:1009F00010918001112319F01130C9F1BFC110927B
:100A00007D0144E06EEF83E50E94730445E560EFED
:100A100082E50E9473048111E6C140E06BEF82E53C
:100A20000E9473048111DFC142E050E0BE016F5F9C
:100A30007F4F8EEF0E94AC048111D5C1898190E077
:100A4000982F88272A81822B90937F0180937E01A3
:100A500081E08093800180937C012FEF4EE954E286
:100A6000215040405040E1F700C0000087C146E0FF
:100A700050E0BE016F5F7F4F80E00E94AC0488238E
:100A800019F010928001AFC1A0917E01B0917F0159
:100A900049819A816E818B81FC81ED81A13071E069
:100AA000B70709F444C0A530B44009F4D8C0042FF6
:100AB000A92FA095262F2C7030E0359527953595D8
:100AC000279544E0849FC0011124282B392B462F01
:100AD000407350E074E0559547957A95E1F774E0DE
:100AE000F79FC0011124482B592BB12FB627B170A5
:100AF00061FFB26080917C01882359F010927C01E3
:100B000080913801B33011F4826001C08D7F8093F1
:100B100038018091380181FD3AC174E0E79FC0013E
:100B200011246295669566956370862B32C1042FF9
:100B3000000F000F24E0929FD0011124A095907C1B
:100B4000292F30E0B5E035952795BA95E1F7407C3F
:100B500050E093E0559547959A95E1F7242B352B76
:100B6000982F991F9927991F292B45E0220F331F92
:100B70004A95E1F7482F4F7170E2479FA001112479
:100B8000409593E05927BE2FB695B695B127B17021
:100B900065FFB26063FFB46066FFB86064FFB06178
:100BA000E5FFB062E1FFB06462FFB068162F1095F8
:100BB0001170E6FF1260E7FF146061FF186067FFC5
:100BC0001061E4FF1062E3FF106460917C01912FDB
:100BD0009074662371F010927C0160913801992322
:100BE00021F06E7F6093380104C06160609338012A
:100BF0001CC09923D1F060917A0170917B01643B14
:100C000071051CF46F5F7F4F0BC0643B710589F465
:100C10009091380161E096279093380165EB70E080
:100C200070937B0160937A0104C010927B01109253
:100C30007A019091380190FDAEC0807690E0959554
:100C4000879595958795F295F695F7708F2B75E0BA
:100C5000880F991F7A95E1F780959095A2C02F2F64
:100C60002C7F50E4259F90011124242B220F331F49
:100C7000220F331F30584E2F4C7F70E4479FA00146
:100C80001124492B440F551F440F551F50586C7F9A
:100C900090E4699FB0011124682B660F771F660FDF
:100CA000771FCB01905860917D016A307CF46F5FB3
:100CB00060937D01309379012093780150937701FF
:100CC000409376019093750180937401609178014F
:100CD00070917901261B370B609176017091770135
:100CE000461B570B6091740170917501861B970B21
:100CF00065E0559547956A95E1F775E09595879577
:100D00007A95E1F7A5E035952795AA95E1F7213089
:100D10006EEF360714F421E03EEF41307EEF5707C7
:100D200014F441E05EEF81306EEF960714F481E039
:100D30009EEF211572E0370714F02FEF31E062E0EB
:100D40003627411572E0570714F04FEF51E062E08B
:100D50005627811572E0970714F08FEF91E062E05B
:100D60009627F1FBBB27B0F961E0B627F0FFB26030
:100D7000E1FFB460E0FF12C0B86010C080E092E014
:100D800040E052E020E032E010E0B0E008C080E057
:100D900092E010E006C080E092E003C010E0A0E81E
:100DA00000E800938901A0938A0120938B01242FEE
:100DB000220F220F232B20938C01282F2295207F96
:100DC00036E0569547953A95E1F7242B20938D010F
:100DD00044E0969587954A95E1F780938E01B0930C
:100DE0008F011093900160960FB6F894DEBF0FBE8E
:100DF000CDBFDF91CF911F910F91089564E380E003
:100E000090E00E94ED090E94EC04389A4098089501
:100E100084EB90E090932B0180932A0186E291E08D
:100E2000089540919F015091A0016091A10170919E
:100E3000A201009729F0FC014083518362837383F0
:100E400040939B0150939C0160939D0170939E0180
:100E50000895EF920F931F93CF93DF9300D0CDB7F8
:100E6000DEB769834A83E12C00E010E020E030E047
:100E7000AE014F5F5F4F62E070E00E94FD09EFEA54
:100E8000F4E03197F1F700C000000F900F90DF9170
:100E9000CF911F910F91EF90089580919A01811148
:100EA00015C090919F0180919B0198130FC0909164
:100EB000A20180919E01981309C080913B01882373
:100EC00019F010923B0102C080E0089581E008957E
:100ED000AF92BF92CF92DF92EF920F931F93CF9377
:100EE000DF931F92CDB7DEB789835B016A01E12CE6
:100EF00000E010E020E030E0AE014F5F5F4F61E0C6
:100F000070E082E50E94FD09811117C08FEA94E02C
:100F10000197F1F700C000008501960140E050E024
:100F200060E070E082E50E94FD09811106C0EFEAF1
:100F3000F4E03197F1F700C000000F90DF91CF91FE
:100F40001F910F91EF90DF90CF90BF90AF900895D9
:100F5000EF92FF921F93CF93DF93CDB7DEB76097E9
:100F60000FB6F894DEBF0FBECDBF109199011123CB
:100F700019F01130B9F1B1C044E06EEF83E50E9481
:100F8000290745E560EF82E50E9429078111EBC141
:100F900040E06BEF82E50E9429078111E4C142E045
:100FA00050E0BE016F5F7F4F8EEF0E946807811196
:100FB000DAC1898190E0982F88272A81822B90932B
:100FC00098018093970181E0809399018093960125
:100FD0002FEF3EE984E2215030408040E1F700C02D
:100FE00000007BC046E050E0BE016F5F7F4F80E0B5
:100FF0000E946807882319F010929901B4C180916A
:1010000097019091980169812A81AE81EB81B0911D
:10101000960181309140F1F0862F422F40952A2F82
:101020002C7030E0359527953595279594E0E99F0C
:10103000F00111242E2B3F2B1A271170A1FF1260F3
:10104000BB2309F452C01092960160933A01409379
:1010500039014BC0862F880F880F34E0239FA001F1
:1010600011244095207C30E095E0359527959A95A0
:10107000E1F7607C70E053E0759567955A95E1F76C
:10108000262B372B9E2F991F9927991F292B65E017
:10109000220F331F6A95E1F7EF71F0E09D8192FF17
:1010A00002C010E001C014E0A5FF1260A3FF1260AF
:1010B000A6FF1160A4FF1160A0FF106196FF1062EF
:1010C00097FF1064A1FF1068BB2389F0109296016E
:1010D00080933A01409339010AC0E0E1F0E020E05A
:1010E00032E010E040E880E802C0E0E1F0E090E0AB
:1010F00050E060913A01861B910960913901461BCD
:101100005109A0919701B09198016091E101109768
:1011100009F085C07091E601772309F448C0209159
:101120009501712F727011FF11C0211112C0262F6D
:1011300030E02417350734F03195219531094217F5
:1011400053073CF421E02093940103C02111109235
:1011500094017093950120919401222329F18091AB
:10116000E301811103C05195419551091D7F809183
:10117000E70190E08417950774F0919581959109A6
:1011800021E030E04817590714F020E030E03195B5
:101190002195310902C021E030E02093930140E025
:1011A00050E080E090E060C0109293015BC032504C
:1011B0007091E301772319F0319521953109E09180
:1011C000E401F0E0E217F30754F42091910130912B
:1011D0009201232B09F52091E50130E012C0F19531
:1011E000E195F1092E173F079CF420919101309170
:1011F0009201232B89F42091E50130E0319521956E
:101200003109E1E0F0E0F0939201E093910127C011
:10121000109292011092910120E030E020C0A130A4
:10122000B14001F570972091E201222319F0F19568
:10123000E195F109E930F1053CF021E030E030932F
:101240009201209391010BC0E83FFF4F0CF721E082
:1012500030E030939201209391012FEF3FEF2093E4
:10126000930102C020E030E070E06817790724F4B1
:10127000FC01E61BF70B0DC0EE27FF27E61BF70B63
:101280008E179F0724F4FC01E60FF71F02C0E0E071
:10129000F0E0641775071CF4461B570B0AC088273B
:1012A0009927861B970B481759070CF058C0460F13
:1012B000571F309751F44115510539F4232B19F478
:1012C000812F807F31F040E050E081E080939A01EF
:1012D00004C010929A0140E050E0E090E001F12C4F
:1012E00014FD06C0CA01B7010E94280C9B0102C070
:1012F0002FEF3FEF15FF02C021E030E016FD05C0E3
:10130000CF01B7010E94280C02C061E070E017FD18
:101310000AC061388FEF78074CF06038710544F0EF
:101320006FE770E005C06FEF7FEF02C061E87FEF0D
:1013300021389FEF390734F0203831052CF02FE7A2
:1013400030E002C021E83FEF10939F016093A001BD
:101350002093A101809193018093A20104C0309752
:1013600009F0B1CFABCF60960FB6F894DEBF0FBED9
:10137000CDBFDF91CF911F91FF90EF90089564E36F
:1013800080E090E00E94ED090E94A807389A4098FA
:1013900008958CE391E00895CF93DF93409AC8EAD3
:1013A000D1E68091BC0087FD10C02197209721F4E1
:1013B00040988FEF9FEF0EC08BE291E00197F1F71D
:1013C00000C000000E940501ECCF40988091B90058
:1013D000887F90E0DF91CF910895892B19F088B133
:1013E000806302C088B18F7C88B96093B800809117
:1013F000B9008C7F8093B90008959F92AF92BF92FD
:10140000CF92DF92EF92FF920F931F93CF93DF93D0
:10141000B82E6B01942EA52E79016115710569F422
:101420002115310539F084EA8093BC000E94CC0973
:1014300097FF39C08FEF9FEF7FC084EA8093BC0095
:101440000E94CC0997FDF6CF883009F071C08B2D32
:10145000880F8093BB0084E88093BC000E94CC0975
:1014600097FDE8CF883109F04FC0C92DDA2DCC0E99
:10147000DD1E24E8A22ECC15DD0569F0899180934C
:10148000BB00A092BC000E94CC0997FDD3CF88324C
:1014900091F323E03EC0E114F10429F684E980933E
:1014A000BC0080E046C0803111F0883079F58B2D8A
:1014B000880F81608093BB0084E88093BC000E9409
:1014C000CC0997FDB7CF803419F5E701219784E85F
:1014D000F82E94ECE92ECF3FFFEFDF07F9F22097CB
:1014E00019F0E092BC0002C0F092BC000E94CC094E
:1014F00097FDA0CF2197877F803581F68091BB0033
:10150000F80181938F01E7CF22E003C024E001C0FE
:1015100025E090E0803A31F0883F69F0883321F48B
:1015200084E803C084EA01C084E98093BC0003C05E
:1015300081E090E001C0822FDF91CF911F910F9148
:10154000FF90EF90DF90CF90BF90AF909F90089565
:10155000E9EDF1E080E090E021E0E83EF207D9F02B
:1015600021919227092E0294202D2F702927392F9F
:101570003025330F307E2327302D3927307F3695A5
:10158000092E000C331F9695969596959F7193277B
:101590009827822FE1CF08950E94A80A9093E9012D
:1015A0008093E80141E150E060E070E089ED91E076
:1015B0000C94730CCF93DF9341E150E060E070E056
:1015C00089ED91E00E94630C8091D9019091DA013C
:1015D0008D3E9E4F91F081E1E9EDF1E0DF011D923A
:1015E0008A95E9F78DEE9EEF9093DA018093D90109
:1015F0000E940A0B0E94CC0A09C0C091E801D09158
:10160000E9010E94A80AC817D90729F7DF91CF91ED
:101610000C942E0B81E390E3A0E3B1E38093DB0114
:101620009093DC01A093DD01B093DE011092DF0105
:1016300084E08093E00185E08093E1011092E20173
:1016400080E88093E4011092E5011092E30181E0CB
:101650008093E60180E48093E70108958091DB01A7
:1016600090E090935101809350018091DC0190E0D3
:1016700090935301809352018091DD0190E090930B
:101680005501809354018091DE0190E090935701C1
:101690008093560108950F931F93DB01082F10E0EC
:1016A000015011090A301105E0F50C5C1F4FF801DB
:1016B0000C943C0C8D919D910D90BC91A02D80932C
:1016C000DB019093DC01A093DD01B093DE0125C026
:1016D0009C919093DF011FC09C919093E0011BC0EF
:1016E0009C919093E10117C09C919093E20113C0EB
:1016F0009C919093E3010FC09C919093E4010BC0E7
:101700009C919093E50107C09C919093E60103C0E2
:101710009C919093E701FA0180830E94CC0A81E0BA
:1017200001C080E01F910F91089517B88FE088B92C
:1017300014B88FEF85B988EF8BB985E08AB914BCEE
:1017400085BD82E08093B00087E08093B10084EC97
:101750008093B3000E94DA0A8091DF01882331F080
:10176000813039F01092DF010E94CC0A0E940807F4
:1017700002C00E94C90990936D0180936C01E091B1
:101780006C01F0916D018481958190937301809338
:10179000720122812093710180859185909370015F
:1017A00080936F01868180936E0120931B011092BC
:1017B0001C010284F385E02D09958BB18A7F8BB9DA
:1017C0008AB185608AB987EC9FEA0197F1F700C07A
:1017D00000008AB18A7F8AB90E9429027894D1E0F8
:1017E000C0E012E0A8950E940501DD2341F0E091E0
:1017F0006C01F0916D010484F585E02D0995B99B8C
:1018000019C0C11115C0E0916C01F0916D01048403
:10181000F585E02D0995E0916C01F0916D0106844C
:10182000F785E02D0995C1E0811103C0C0E001C03A
:10183000C1E017BBC11102C0D0E0D4CF8091AE018E
:1018400084FD02C0C1E0F8CF0E942304C0E0F4CFC1
:1018500097FB072E16F4009407D077FD09D00E945D
:10186000420C07FC05D03EF4909581959F4F08955A
:10187000709561957F4F0895EE0FFF1F0590F491CD
:10188000E02D0994AA1BBB1B51E107C0AA1FBB1F77
:10189000A617B70710F0A61BB70B881F991F5A95FC
:1018A000A9F780959095BC01CD010895FB01DC015D
:1018B00004C08D910190801921F441505040C8F727
:1018C000881B990B0895DC01CB01FC01F999FECF2F
:1018D00006C0F2BDE1BDF89A319600B40D924150B8
:1018E0005040B8F70895DC01A40FB51F4150504097
:1018F00048F0CB01840F951F2E910E94840C41501B
:101900005040D0F70895262FF999FECF92BD81BDA2
:10191000F89A019700B4021639F01FBA20BD0FB62D
:0E192000F894FA9AF99A0FBE0895F894FFCF42
:10192E00FF5A0902220001010000320904000001E1
:10193E0003000000092101010001220000070581BA
:10194E000308000A010008005500000012000901FA
:10195E00FE06EC0497045F0401808001040055002C
:10196E002D0112001B01BF09A8074D0711070A031D
:08197E0032003000300030009F
:00000001FF
